:102CB40033302E32202020000001FF00FF000001ED
:102CC400010000FF00FF01001020304050607080C0
:102894004102720041027900410277004102740052
:1028A4004102AC00C103C18BC108C18DC109C1047F
:1028B400C10CC107C10A43020B00002441020200FB
:0428C4004102A3200A
:1023F200E4900273F0D20BD20DD206D201D205D2F2
:10240200009002ACE0243CF582E43402F583E4F06F
:10241200900274E02444F582E43402F583E4F090FF
:102422000272E0240EF582E43402F583E4F09002B5
:1024320077E02403F582E43402F583E4F07F289008
:10244200027A7401F0A3DFFC7F0490020F7401F0A2
:10245200A3DFFC7F079002047401F0A3DFFC7F2856
:102462009002B77401F0A3DFFC7F0490024574016F
:0F247200F0A3DFFC7F0790023D7401F0A3DFFCB5
:012481002238
:031A24000218CED7
:1018CE00C0E0C0F0C083C082C0D075D000C000C0E0
:1018DE0001C002C003C004C005C006C007C2DF209D
:0518EE00DA0330DB68A5
:1018F3009003ECE5A0F0C2DBC2DA9002FFE0FF90B8
:1019030003ECE0FE6F540C604FEE13135403FDEF32
:10191300540CFF7E00ED4F24BCF582EE342CF5838E
:10192300E493FF9003EDF09002A2E0FE9003EEF04B
:101933009002A22FF0E06E30E1169003EDE07F04F9
:10194300B40105122B218003122DB3D20C122DE406
:081953009003ECE09002FFF0AC
:06195B0020D80330D9740E
:101961009003ECE5A0F0C2D9C2D8900249E0FF9003
:1019710003ECE0FD6F5403605BEF75F004A47E009F
:10198100540CFFED5403FDEF4D24BCF582EE342CD5
:10199100F583E493FF9003EDF090023BE0FE9003AA
:1019A100EEF090023B2FF0E06E30E1209003EDE08D
:1019B1007F04B40105121FE080031222119002730B
:1019C100E0FFE4FD121EE0D20C122DE49003ECE0E6
:0419D100900249F047
:1019D500D007D006D005D004D003D002D001D00066
:0B19E500D0D0D082D083D0F0D0E03210
:102D4B0075DA3175DB3175DC3175DD31E49002A25A
:0A2D5B00F043F61075D982D2DE2293
:102E3F0075BC4075E8C075BA1F75D108E4F5BB4382
:032E4F00E6082270
:0A2ED70075A14075F80175A20722ED
:092EFF00E4F5B1F5A975B28322D6
:0D2E8F0075921E7593FF75910443E6802235
:0D2E7300E4FF74242FF876FF0FEFB428F56C
:012E8000222F
:102A810078AC7C037D017BFF7A2C79CC7E007F08BA
:102A91001213FDE4FFEF75F0058424ACF582E434F4
:102AA10003F583E0FE74132FF582E43402F583EE1F
:062AB100F00FEFB428DF76
:012AB70022FC
:102D130075A4CDE4F5F275F3FF75D4C875D5FF75C9
:0C2D2300F41F75A70175E10675E244225B
:0D2E8100E4FF744C2FF8E4F60FEFB428F5D1
:012E8E002221
:0A2EB6007F109002ADE4F0A3DFFCF2
:012EC00022EF
:102E1300758850758922758E0C758AAE758CAE7562
:062E23008BC7758DC7226C
:102C1000E4F5D9122EFF122D131223F2122E3F12B9
:102C20002E8F122D4B122ED7122A81122EB6022E63
:012C30001390
:102DB300900278E0244CF8E6FED394045004E4F641
:092DC3008004C3EE9FF6022A44CD
:102B2100900278E0FE244CF8E6FDEF2DFDE433FC45
:102B3100C3ED94FFEC648094804008744C2EF876C9
:102B4100FF800A900278E0244CF8EF26F6022A442E
:101FE0009003EFEFF090020BE0FBA3E0FAA3E0F91F
:101FF000900273E0F58275830012143CB4FF1990CF
:102000000273E0FF2424F876E3744A2FF582E43467
:1020100002F58374E30220A290020BE0FBA3E0FA36
:10202000A3E0F9900273E0F58275830012143CD3AB
:1020300094035017900273E0FF2424F8E4F6744AE6
:102040002FF582E43402F583E4805790020BE0FB25
:10205000A3E0FAA3E0F9900273E0FFE92FF9E43A74
:10206000FA121423FE9003EFE0FDC3EE9D12149CC0
:1020700090020BE0FBA3E0FAA3E0F98F82758300E6
:1020800012143CFF900273E0FE2424F8A6078E820F
:1020900075830012143CFF744A2EF582E43402F575
:0720A00083EFF0122A042275
:102211009003EFEFF090020BE0FBA3E0FAA3E0F9EB
:10222100900273E0F58275830012143CC394E3407D
:1022310018900273E0FF2424F876FF744A2FF58288
:10224100E43402F58374FF807290020BE0FBA3E09B
:10225100FAA3E0F9900273E0F58275830012143C51
:102261007018900273E0FF2424F87603744A2FF566
:1022710082E43402F583740380419003EFE0FF9020
:10228100020BE0FBA3E0FAA3E0F9900273E0FEF594
:1022910082758300EF1214698E8275830012143CDB
:1022A100FF74242EF8A6078E8275830012143CFF5A
:1022B100744A2EF582E43402F583EFF0122A0422E7
:102E2900900278E0244CF8E6700476FF8002E4F61C
:062E3900122A44022DE400
:1026270090020BE0FBA3E0FAA3E0F9900273E0FF4E
:10263700F58275830012143CB4FF098F82758300FD
:102647007423801690020BE0FBA3E0FAA3E0F99055
:102657000273E0F58275830074FF1214AE90020BCB
:10266700E0FBA3E0FAA3E0F9900273E0FFF58275BF
:10267700830012143CFE74242FF8A606900273E020
:10268700FFF58275830012143CFE744A2FF582E42D
:102697003402F583EEF0122A04900273E0FFE4FDA2
:0626A700121EE0022DE40A
:041EDC007D01E4FFA1
:051EE0009003EFEFF09C
:101EE500E49003F4F0C212C21353E6EFEDB4010817
:101EF500D2129003EF7427F0EDB40206D213C2B0EC
:101F05008002D2B09003EFE0FD75F00584E5F004A2
:101F15009003F2F0ED75F0058404A3F0D287C28634
:101F25009003F17408F0C283122F08301303021FC7
:101F3500BC9003F07405F09003F0E0FFC3940140FA
:101F4500769003F3E0FE9003F1E0FDB50607A3E00C
:101F5500FEEF6E600330124D90020BE0FBA3E0FA3A
:101F6500A3E0F99003EFE0F58275830012143CC4F9
:101F7500540FFFEDC454F04FFF122F1090020BE0E9
:101F8500FBA3E0FAA3E0F99003EFE0F58275830087
:101F950012143CC454F0FF122F103012129003EFAC
:101FA500E014F0800AE4FF122F10E4FF122F1090C6
:101FB50003F0E014F08080A2139214122786122FEA
:101FC50008D2839003F1E014F0E0C39401400302CA
:0A1FD5001F2B122F08C2B043E610C4
:011FDF0022DF
:072F0800E4FF0FEFB464FBCE
:012F0F00229F
:082F1000E5A120E7FB8FA322DD
:10278600201405E4FF122F10900202E04430FF12DD
:102796002F10E025E024ADF582E43402F583E0C491
:1027A600F854F0C8A3E0C4540F48FF122F1090024B
:1027B60002E025E024ADF582E43402F583A3E0C40B
:1027C600F8540FC868FF0582D58202158315821258
:0D27D6002F10900202E004F0B40502E4F0C0
:0127E30022D3
:072F28007D02E4FF021EE040
:100C9D009003AC7401F053E6EFC2B0C287D286C2A6
:100CAD0083122F089003ACE0FF700302108314B47D
:100CBD000E0050F0900CCF75F003A4C58325F0C540
:100CCD008373020CF9020D3A020D77020DC1020D6C
:100CDD00E5020E09020E4F020E89020ED3020F1A03
:100CED00020F5A020FA1020FE702103290029BE091
:100CFD0025E0FF9002A0E04F25E0FF90029AE04F23
:100D0D0025E0FF90029FE04FF9E4FCFD74442DF5C2
:100D1D008274023CF583E0FFE925E0FEEF4EF90D0C
:100D2D00BD00010CED64044C70E2020F9E9002991F
:100D3D00E025E0FF90029EE04F25E0FF900298E055
:100D4D004F25E0FF90029DE04F25E0FF9002C6E0A9
:100D5D004F25E0FF9002C1E04F25E0FF9002BCE07F
:100D6D004F25E0FF9002B7020ECF900293E025E0F1
:100D7D00FF90028EE04F25E0FF900289E04F25E0C5
:100D8D00FF900284E04F25E0FF9002DAE04F25E06E
:100D9D00FF9002D5E04F25E0FF9002D0E04F25E017
:100DAD00FF9002CBE04FF9FF122F109003ACE0043F
:100DBD00F0020CB1E4FCFD743C2DF58274023CF59F
:100DCD0083E0FFE925E0FEEF4EF90DBD00010CEDCE
:100DDD0064084C70E2020F9EE4FCFD74032DF58255
:100DED0074023CF583E0FFE925E0FEEF4EF90DBD01
:100DFD0000010CED64084C70E2020F9EE4FCFD74E2
:100E0D000E2DF58274023CF583E0FFE925E0FEEF3F
:100E1D004EF90DBD00010CED64054C70E27C007DBA
:100E2D0002747A2DF58274023CF583E0FFE925E02A
:100E3D00FEEF4EF90DBD00010CED64054C70E202A4
:100E4D000F9E90027BE025E0FF90027AE04F25E0B7
:100E5D00FF900282E04F25E0FFA3E04F25E0FF90D9
:100E6D000281E04F25E0FF900280E04F25E0FF90EA
:100E7D00027FE04F25E0FF900288804690028DE0D2
:100E8D00F97C007D0B747A2DF58274023CF583E0BC
:100E9D00FFE925E0FEEF4EF90DBD00010CED640EEE
:100EAD004C70E2E925E0FF90028CE04F25E0FF90C9
:100EBD00028BE04F25E0FFA20BE4334F25E0FF90BE
:100ECD00028AE0020F557C007D15747A2DF582742F
:100EDD00023CF583E0FFE925E0FEEF4EF90DBD0084
:100EED00010CED64194C70E27C007D1D747A2DF5BA
:100EFD008274023CF583E0FFE925E0FEEF4EF9ED4B
:100F0D001D70011CED64194C70E2020F9EA206E4E7
:100F1D003325E0FFA201E4334F25E0FF90029CE072
:100F2D004F25E0FF9002A1E04F25E0FF900248E041
:100F3D004F25E0FFA20DE4334F25E0FFA205E4337A
:100F4D004F25E0FFA200E4334FF902102B7C007D0A
:100F5D000174B72DF58274023CF583E0FFE925E0BD
:100F6D00FEEF4EF90DBD00010CED64054C70E27CF9
:100F7D00007D0674B72DF58274023CF583E0FFE920
:100F8D0025E0FEEF4EF90DBD00010CED640A4C702D
:100F9D00E202102B7C007D0B74B72DF58274023CA0
:100FAD00F583E0FFE925E0FEEF4EF90DBD00010CE4
:100FBD00ED640F4C70E27C007D1374B72DF58274D7
:100FCD00023CF583E0FFE925E0FEEF4EF9ED1D70E3
:100FDD00011CED640F4C70E280447C007D1574B7EC
:100FED002DF58274023CF583E0FFE925E0FEEF4E1E
:100FFD00F90DBD00010CED64194C70E27C007D1DF6
:10100D0074B72DF58274023CF583E0FFE925E0FE0F
:10101D00EF4EF9ED1D70011CED64194C70E290035B
:10102D00ACE00480487C007D1F74B72DF5827402FE
:10103D003CF583E0FFE925E0FEEF4EF90DBD000123
:10104D000CED64234C70E27C007D2774B72DF58286
:10105D0074023CF583E0FFE925E0FEEF4EF9ED1D4E
:10106D0070011CED64234C70E2E49003ACF0AF0111
:0E107D00122F10020CB1D28343E610022F088E
:0B22C1009003F0EEF0A3EFF030086097
:1022CC009003F0A3E0FF122F189003F2EFF09002AE
:1022DC0077E075F005A42F9003F3F09003F0A3E0E2
:1022EC00FF122EC1EF75F007A4FF9003F2F09002DD
:1022FC000BE0FBA3E0FAA3E0F99003F3E0F58275A1
:10230C00830012143CD39F40047F0180027F009015
:0F231C0003F0A3E0247AF582E43402F583EFF0B6
:10232B002290020BE0FBA3E0FAA3E0F99003F0E0AC
:10233B00FEA3E0FFF5828E8312143CB4FF047D01F3
:10234B0080027D00747A2FF582E43402F583EDF080
:01235B00225F
:102D2F00AD07744C2DF8E670047C0180027C0074B2
:0C2D3F00B72DF582E43402F583ECF0229D
:102A040090020BE0FBA3E0FAA3E0F9900273E0FF6D
:102A1400F58275830012143CFEB4FF06D201D2067F
:102A24008019EE7006D201C2068010EED3942340C2
:102A340006C201D2068004C201C2067E000222C17F
:102A4400900278E0FF244CF8E6FE7011D200D20523
:102A540074B72FF582E43402F5837401F0EED39455
:102A6400004013C200D205900278E024B7F582E456
:0C2A74003402F583E4F0EEB4FF02C2056A
:012A80002233
:0A2EC100EF75F0058475F005A4FF1D
:012ECB0022E4
:082F1800EF75F00584AFF02213
:1027E400C20BE4FD7C2890024A74FFF0A3DCFCEFEA
:1027F4003395E0FE7C007D051214D0AC06AD07EFE6
:102804002405FBE43EFAC3ED9BEA6480F8EC6480A3
:1028140098501974242DF8E6FB744A2DF58274023D
:102824003CF583EBF00DBD00010C80D390020B74DA
:0A28340001F0A37402F0A3744AF04F
:01283E002277
:102E6300D20B90020BE4F0A37400F0A37424F022BD
:10108B00E49003ADF07B017A0379AE122B51EF7034
:10109B000302132C9003B0E012156F111704115EAD
:1010AB000510D91410C51610D01710DE1A11001B1D
:1010BB00110B1D11111E000011AED209C20DC21968
:1010CB00D20C0211AEC209D20DD20C0211AED20358
:1010DB000211AE7B017A0379AE9003BEEBF0A3EA6B
:1010EB00F0A3E9F0121423FE9002A3E0FF6E60035D
:1010FB000211AE80059002A3E0FF122C730211AE19
:10110B00122F360211AE122F3D0211AE7B017A0364
:10111B0079AE9003C1EBF0A3EAF0A3E9F0900003E2
:10112B0012143CFF9002A3E06F707830096D9003AE
:10113B00C104F0A3EAF0A3E9F090000512143CFF00
:10114B0090000612143CFD90000412143CFB122379
:10115B005C80487B017A0379AE9003C1EBF0A3EA84
:10116B00F0A3E9F090000312143CFF9002A3E06F90
:10117B0070313009269003C104F0A3EAF0A3E9F023
:10118B0090000512143CFF90000612143CFD9000D9
:10119B000412143CFB1220A7122B7D9002A3E0FF3C
:1011AB00122CF42009030212999003B0E01460355D
:1011BB0024FA6058147003021264240660030212AE
:1011CB0099122E527B017A0379AE9003BEEBF0A3FA
:1011DB00EAF0A3E9F090000312143C900352F012D2
:1011EB002F43021296122E527B017A0379AE900393
:1011FB00BEEBF0A3EAF0A3E9F090000312143C90CD
:10120B000352F09003AD7401F0021296122E527B32
:10121B00017A0379AE9003C4EBF0A3EAF0A3E9F0F3
:10122B0090000312143CFF90000412143CFD90003C
:10123B000512143CFBC0039003C4E0FBA3E0FAA32C
:10124B00E0F990000612143C9003CAF0D00312216F
:10125B005D9003AD7401F08032122E527B017A0344
:10126B0079AE9003C4EBF0A3EAF0A3E9F09000038E
:10127B0012143CFF90000412143CFD900005121454
:10128B003CFB12175C9003AD7401F0122EEB900334
:10129B00ADE06401600302132C122B7D7F289002BA
:1012AB004A74FFF0A3DFFC900277E075F005A4FE13
:1012BB00FFEE2405FDE433FCEFC39DEC6480F87472
:1012CB008098501574242FF8E6FD744A2FF582E4AC
:1012DB003402F583EDF00F80D8E49003ACF090036B
:1012EB00ACE0FFC39428500D7E001222C19003ACDA
:1012FB00E004F080E9E49003ACF09003ACE0FFC3B2
:10130B009428500D7E00122D2F9003ACE004F0803A
:10131B00E9122A04122A44D20C121EDCE49003AD0B
:01132B00F0D1
:01132C00229E
:1008A700122C109002A3E0FF122EA943F601122D7D
:1008B70099E4900352F0122B7DD2AFE49003A7F096
:1008C7009003A7E0FFC39428500D7E001222C19029
:1008D70003A7E004F080E9E49003A7F09003A7E002
:1008E700FFC39428500D7E00122D2F9003A7E0041C
:1008F700F080E9122A04122A44C208C209D20CC2A3
:10090700B0121EDC53E6EFE5147003020AA924FEB9
:1009170070030209EB24FA7003020A2D24F870030E
:10092700020A4E240C6003020A82900277E0FF2439
:1009370003F582E43402F5837401F0900279EFF055
:10094700900277E004F0E0D394074002E4F09002CD
:1009570077E0FF2403F582E43402F583E4F0EF75D2
:10096700F005A4FF900272E02FFFA3F07E00122291
:10097700C1200803020A28E49003A4F09003A4E02E
:10098700FFC394285015744A2FF582E43402F58387
:1009970074FFF09003A4E004F080E1900277E07523
:1009A700F005A49003A5F09003A4F09003A5E0241C
:1009B70005FFE433FE9003A4E0C39FEE6480F87460
:1009C7008098501BE0FF2424F8E6FE744A2FF58236
:1009D700E43402F583EEF09003A4E004F080CC1237
:1009E7001EDC803D900272E0240EF582E43402F5AD
:1009F700837401F0900272E004F0E0D394044002A3
:100A0700E4F0900272E0FF240EF582E43402F583ED
:100A1700E4F0900277E075F005A4FEEF2E900273E4
:100A2700F0122A04805520030CE4900352F0122F91
:100A370043D20D8046A209B39209300906C219C2F2
:100A47000D8038D20D8034A208B3920830080A907E
:100A57000277E0FF1227E48003122E63E49003A5D8
:100A6700F09003A5E0FFC39428500D7E001222C129
:100A77009003A5E004F080E9121EDC30081FE49023
:100A870003A5F09003A5E0FFC39428500D7E001244
:100A970022C19003A5E004F080E9121EDCE4F514FE
:100AA700D20CE5137003020B4E24E0601524E060BE
:100AB7005124C0601224706003020B4912262702DA
:100AC7000B49122E29807B9002ACE0243CF582E48E
:100AD7003402F5837401F09002ACE004F0E0D394A3
:100AE700074002E4F09002ACE0FF243CF582E434D6
:100AF70002F583E4F0EF75F005A4FF900274E02F90
:100B07008039900274E02444F582E43402F583745A
:100B170001F0900274E004F0E0D394044002E4F0A2
:100B2700900274E0FF2444F582E43402F583E4F094
:100B37009002ACE075F005A4FEEF2E900278F0125B
:100B47002A44D20CE4F51330081CE49003A5F09076
:100B570003A5E0FFC39428500D7E001222C1900325
:100B6700A5E004F080E9200203020C6CC20243E610
:100B770010E49003A4F09003A812153E00000000B3
:100B8700E49003A6F09003A8E0F8A3E0F9A3E0FA45
:100B9700A3E0FBC0009003A4E0FF9003A6E0FE756E
:100BA700F005A42F244CF8E6FF74A42EF582E43454
:100BB70002F583E0FEEF8EF0A4FFE4FCFDD000EB2E
:100BC7002FFFEA35F0FEED39FDEC38FC9003A81253
:100BD70015329003A6E004F0E0B408A9E47FFF7E95
:100BE700FFFDFC9003A8E0F8A3E0F9A3E0FAA3E077
:100BF700FBD312150E400A9003A812153E0000FF02
:100C0700FF9003A8E0FCA3E0FDA3E0FEA3E0FF78CC
:100C17000412151F9003A4E0FD25E024ADF582E43E
:100C27003402F583EEF0A3EFF0ED25E024ADF58275
:100C3700E43402F583E0FEA3E0C394FFEE940F4093
:100C470013ED25E024ADF582E43402F583740FF04B
:100C5700A374FFF09003A4E004F0E06405600302CE
:100C67000B7D122F2812108B3007109002A3E0FF84
:100C77007BFF7A2C79B4122726C207300A0A900222
:100C8700A3E0FF122C52C20A200C0302090B120C1C
:060C97009DC20C02090BD6
:10259D00E5B0541EF512650E600CE512650EF516CC
:1025AD0075113285120EE51160431511E511703D5F
:1025BD00E51630E108E51220E103751402E5163049
:1025CD00E208E51220E203751404E51630E311E587
:1025DD001220E30C900275740BF0A374B8F0D20EB8
:1025ED00E51630E408E51220E403751410300E29C9
:1025FD00900276E024FFF0900275E034FFF0E5B034
:10260D0030E305751408C20E900275E07002A3E068
:0A261D007007C20E300302D207223C
:10283F00E5A054F0F510650D600CE510650DF5156C
:10284F00750F3285100DE50F603A150FE50F7034D7
:10285F00E51530E408E51020E403751310E5153095
:10286F00E508E51020E503751320E51530E608E5CA
:10287F001020E603751340E51530E708E51020E753
:05288F00037513802217
:031A2D00022C94F4
:102C9400C0E0C083C082C0D053917F12259D12280A
:102CA4003F75BB0075E8D0D0D0D082D083D0E0325D
:031A210002292E69
:10292E00C0E0C083C082C0D075D000C006C007C250
:10293E00EDE5BB64086025E5BEC4333354C0FFE546
:10294E00BD1313543F4FFFAEBB74A42EF582E43477
:10295E0002F583EFF005BB75E8D08002D202D007F6
:0B296E00D006D0D0D082D083D0E03261
:1028C800420350000042030B00004203060000C10F
:0528D80018C117C11634
:0A2EE100C217C218E490030AF022A1
:102BCB00E4900350F0A3F090030BF0A3F0A3F0906C
:102BDB000306F0A3F0900301F0A37430F0E490032C
:032BEB0009F022CC
:061A1B00122EE1022BCBAC
:0D2E9C0075C19043E6019003087401F02217
:102E520043C140E5C120E5FB121A1BE4900308F0D0
:012E6200224D
:0A2EEB0053C1BF9003087401F022E8
:0D2EA900AE07122E9C900305EEF0021A1BDE
:102BA600E49003D8F0A3F0301702FF222018FDD2DC
:102BB60017900303E4F0A37410F090033EEFF0E4E3
:042BC600A3F07F01F8
:012BCA0022E8
:102AED0030170A900303E07002A3E070037F002209
:102AFD00900304E024FFF0900303E034FFF0900313
:102B0D003FE0FE04F074402EF582E43403F583EFCC
:042B1D00F07F012222
:0B2ECC00301707C217D218122EF52293
:0A2EF500E5C120E5FBC2C4D2C522EE
:1026AD009003D2EBF0A3EAF0A3E9F0900308E070F9
:1026BD0002FF229003D5E0FE6005D3941040037F06
:0826CD000022122BA6EF604E63
:1026D500E49003D7F09003D5E0FF9003D7E0FEC365
:1026E5009F50249003D2E0FBA3E0FAA3E0F98E8289
:1026F50075830012143CFF122AEDEF7002FF229041
:1027050003D7E004F080CEE490030AF0122ECC90BB
:0E27150003D6E070032018FD90030AE0FF22B7
:032723007FFF2213
:0E1CCA009003CAEBF0A3EAF0A3E9F0A3EDF05B
:101CD800E4FFD3900351E09400900350E0648094B3
:101CE8008050012253E6FE900306E0FEA3E0240D97
:101CF800F58274033EF583E0FF900306E475F00176
:101D08001214E2FCE5F064304C7006900306F0A370
:101D1800F0900302E004F07006900301E004F0E4A0
:101D2800FE9003CDE0FDEEC39D5054EEC39F504F8F
:101D3800900306E0FCA3E0240DF58274033CF583D0
:101D4800E0FD9003CAE0FBA3E0FAA3E0F98E8275F8
:101D58008300ED1214AE900306E475F0011214E24C
:101D6800FCE5F064304C7006900306F0A3F0900395
:101D780002E004F07006900301E004F00E80A2EE89
:101D8800C39F5029900306E475F0011214E2FCE5A4
:101D9800F064304C7006900306F0A3F0900302E064
:101DA80004F07006900301E004F00E80D290035115
:101DB800E024FFF0900350E034FFF043E601900385
:0C1DC800CDE0FEEFC39E50028002AF068B
:011DD40022EC
:102DCC00D3900351E09400900350E06480948040D1
:082DDC00047F0180027F002248
:031A18000215C1F3
:1015C100C0E0C0F0C083C082C0D075D000C000C0F0
:0315D10006C0074A
:1015D400C215E5C054FE12156F16B00816B00A16EF
:1015E400770C16770E172910172912167D221688E4
:1015F4002816882A167D2C167D2E166AC01623C23C
:10160400160EE0160EE200001734C21690033EE0F8
:10161400F5C2C2C5C2C490033D74FFF002173690F0
:10162400033DE0FFB4FF1290033FE0F5C2C2C5C220
:10163400C490033DE4F002173690033FE0FEEFC38D
:101644009E501790033DE0FF04F074402FF582E4B0
:101654003403F583E0F5C2021736D2C490030AE4DA
:10166400F0C21802173690030A74FDF0D2C5C2C442
:1016740002173690033D74FFF0D216C2C4C2C1D221
:10168400C5021736E5C26007900305E0B5C20E90A7
:101694000300E4F0C2C5C2C4D2C1021736C2C4C238
:1016A400C130160302172EC2C5021736900300E09C
:1016B4007020E5C2F0E0FFC3900302E09F7480F85D
:1016C400900301E06480985003122BCB900300E058
:1016D40004F0900302E024FFF0900301E034FFF0F3
:1016E40090030BE0FEA3E0240DF58274033EF58322
:1016F400E5C2F090030BE475F0011214E2FEE5F08C
:1017040064304E700690030BF0A3F0900300E014D5
:10171400F0700E900351E004F07006900350E00462
:10172400F0D2C1800DC2C4301608C216D2C58002E0
:10173400D21530151053C17F43C180C2C5C2C4C283
:07174400C1C215C218C2C0AA
:10174B00D007D006D000D0D0D082D083D0F0D0E05C
:01175B00325B
:051A2700E5C15420FFA1
:011A2C002297
:072F2F0043C14053E6FE22FE
:101A30009003D8E0FFA3E0FCA3E0FDA3E0FBA3E05C
:101A4000FAA3E0F99003E7E517F0E518A3F0900397
:061A5000E0E09003E9F064
:101A56009003E1EFF0A3ECF0A3EDF0A3EBF0A3EA23
:041A6600F0A3E9F010
:101A6A009003EA7403F0A374E8F0E5C120E5FBD221
:101A7A00C1C2C4D2C5E4FF9003F6F030C0FDE5C090
:101A8A0054FE24407003021B2D24FE602424E260CD
:101A9A000924FE600524E2021B35C2C5EF60030279
:101AAA001B3B9003E1E025E044A0F5C27F03021B43
:101ABA003BEFB4030A9003E2E0F5C27F058072EFC0
:101ACA00B4050B9003E2A3E0F5C27F068063EF64DE
:101ADA0006703E9003E9E09003E4700FE0FBA3E494
:101AEA0075F0011214F8A9F0FA8008E0FBA3E0FAF5
:101AFA00A3E0F9121423F5C29003E8E024FFF09062
:101B0A0003E7E034FFF0E07002A3E070247F07806F
:101B1A0020EFB40706D2C47F0980169003F6740535
:101B2A00F0800E9003F67402F080069003F67401BA
:101B3A00F0EFB40904C2C080369003F6E0FE6406F2
:101B4A006012EEB402169003EA74FFF5F01214E282
:101B5A0045F06008D2C5E49003F6F0FF9003F6E082
:101B6A006008C2C5D2C4C2C08005C2C0021A85E5D7
:041B7A00C120E5FBA6
:011B7E002244
:101B7F009003D9EFF0A3ECF0A3EDF0A3EBF0A3EA01
:041B8F00F0A3E9F0E6
:101B93009003E17403F0A374E8F0E5C120E5FBD200
:101BA300C1C2C4D2C5E4FF9003F6F030C0FDE5C066
:101BB30054FE24C87003021C7024AE607A24CA70D9
:101BC30003021C7824FE603824E2600924FE6005C9
:101BD30024E2021C80C2C5EF700F9003D9E025E018
:101BE30044A0F5C27F03021C86EF64016003021C5C
:101BF300869003D9E025E044A1F5C27F04021C8648
:101C0300EFB4030A9003DAE0F5C27F058075EFB401
:101C1300050B9003DAA3E0F5C27F068066EFB406F6
:101C230006D2C57F01805CEFB404047F0280549028
:101C330003F67405F0804C9003DCE0FBA3E475F03D
:101C4300011214F8A9F0FAE5C212149C9003E0E023
:101C530024FFF09003DFE034FFF0E07002A3E070B4
:101C6300087F09C2C1D2C4801A7F0280169003F68E
:101C73007406F0800E9003F67402F080069003F66B
:101C83007401F0EFB40904C2C080369003F6E0FE9D
:101C930064066012EEB402169003E174FFF5F012CD
:101CA30014E245F06008D2C5E49003F6F0FF900318
:101CB300F6E06008C2C5D2C4C2C08005C2C0021B20
:061CC300AEE5C120E5FBC7
:011CC90022F8
:101DD5009003D8EFF09003DBEBF0A3EAF0A3E9F072
:081DE5009003D9ECF0A3EDF02E
:101DED00751900543FF51A543F605CC37440951A41
:101DFD00FFE49519FE9003DEE0FCA3E0FDC39FEC2C
:101E0D009E50068C178D1880048E178F18121A305D
:101E1D009003F6E060037F02229003DAE02518F0CC
:101E2D009003D9E03517F09003E0E0700B9003DCE0
:101E3D00E5178518F01214E2C39003DFE09518F052
:101E4D009003DEE09517F09003DEE0F517A3E0F5C3
:101E5D0018D3E5189400E51794004070E5189440E8
:101E6D00E51794005013121A309003F6E060037FCB
:101E7D000222E4F517F51880D89003D8E0FFA3E00F
:101E8D00FCA3E0FDA3E0FBA3E0FAA3E0F99003E7D8
:101E9D00E4F07440121A4C9003F6E060037F0222C6
:101EAD0074C02518F51874FF3517F5179003DAE08F
:101EBD002440F09003D9E03400F09003E0E07091FD
:0E1ECD009003DC75F0401214E2021E5E7F00EE
:011EDB0022E4
:102DFC009003DFE4F0A304F0121B7F9003F6E06075
:072E0C00037F01227F002279
:102D65009003F5EBF07B017A0379F59003DEE4F04F
:0A2D7500A304F0E4A3F0121DD52220
:102BEE00C0079003D7E0FFA3E09003DFCFF0A3EF81
:102BFE00F0D007121B7F9003F6E060037F01227F67
:022C0E000022A2
:102D7F00C0079003D6E0FFA3E09003DECFF0A3EFF0
:0A2D8F00F0E4A3F0D007121DD522D6
:102C3100A2AFE433FCC2AF758F0175B7A575B7F1CB
:102C41008F828E83EDF0E4F58FAF04EF24FF92AF16
:012C51002260
:102CD400A2AFE433FDC2AF758F0375B7A575B7F125
:0F2CE4008F828E83E4F0F58FAF05EF24FF92AF60
:012CF30022BE
:1028E2009003DEEEF0A3EFF0A3ECF0A3EDF0EB4AE1
:1028F20060399003DEE0FEA3E0FFA3E0FCA3E0F575
:10290200828C83E0FD122C31EB1B70011A9003E1E3
:10291200E004F070069003E0E004F09003DFE004CE
:0C292200F070CB9003DEE004F080C322D4
:082F2000E4900000F0A3F02290
:1019F000900000E0FEA3E0FF122CD4900000E0FE77
:101A0000A3E0FF7C007D027B007A021228E2E490D2
:061A10000000F0A3F0222B
:0A251100A9059003D8EEF0A3EFF047
:10251B00EE54FEFE900000E0FCA3E0FD7002EE6CBA
:10252B006057ED4C60031219F09003D8E0FEEE54A7
:10253B00FEFE7F00900000F0A3EFF09003DAEEF0C8
:10254B00A3EFF0A37400F0A37402F07E029003DA01
:10255B00E475F0011214F885F082F583E493FD9095
:10256B0003DCE475F0011214F885F082F583EDF0CD
:10257B00EF1F70011EEF4E70D49003D8E0FCA3E068
:10258B00FDEC5401FC74022DF58274003CF583E9DB
:01259B00F04F
:01259C00221C
:102979009003D1EEF0A3EFF0A3EBF0A3EAF0A3E903
:10298900F09003D674FFF5F01214F845F060269024
:1029990003D1E475F0011214F8AFF0FE9003D3E00F
:1029A900FBA3E475F0011214F8A9F0FA121423FD3F
:0629B90012251180CC2262
:0E29BF009003CBEBF0A3EAF0A3E9F0A3EDF058
:1029CD00E49003D0F09003CBE0FBA3E0FAA3E0F991
:1029DD00A3E09003D5F09003CFE09003D6F0E4FF91
:1029ED001226ADEFB4FF0D9003D0E0FE04F0EEC360
:0629FD00940340D17E00AE
:012A030022B0
:0B2B51009003C7EBF0A3EAF0A3E9F04B
:102B5C007E007F007D101215959003C7E0FBA3E06B
:102B6C00FAA3E0F97D10121CCAEF7002FF227F015C
:012B7C002236
:102726009003AC7422F0A3EFF0A37413F0121423F9
:102736009003AFF090000112143C9003B0F09000AB
:102746000212143C9003B1F090000312143C900363
:10275600B2F090000412143C9003B3F090000512FE
:10276600143C9003B4F090000612143C9003B5F0AC
:102776007B017A0379ACE49003CFF07D0A0229BF8E
:102C52009003AC7422F0A3EFF0A37403F0A374FF0B
:102C6200F07B017A0379ACE49003CFF07D04022972
:012C7200BFA2
:102C73009003C77422F0A3EFF0A3741CF0A374FFB6
:102C8300F07B017A0379C7E49003CFF07D04022936
:012C9300BF81
:102CF400E49003C7F0A3EFF0A3740AF0A3EFF07B12
:0F2D0400017A0379C7E49003CFF07D040229BF61
:0428DD004103A30010
:062F3D00E49003A3F02262
:072F36009003A37401F022D7
:102482009003AC7403F0E4A3F0A3F0122F207E3B80
:102492007F607B017A0379AC9003D6E4F0A304F069
:1024A2001229791219F07E007F507D007B007A009C
:1024B2007924121595122E73122E81E49003ADF039
:1024C2009003ADE0FFC3941E502A75F050EFA42490
:1024D20000F582E5F03432AF82FE7B007A00792487
:1024E2009003D6E4F0A37450F01229799003ADE082
:1024F20004F080CC1219F07E3B7F617B017A037974
:0F250200AE9003D6E4F0A304F01229790219F089
:102DE40020191430030D30090C9003A3E07006D2AF
:082DF4000A8002C20DD219226F
:102D9900903B61E493F46009903B60E493640360C1
:0A2DA90003122482E4900352F0228A
:102B7D00900352E0FFC3941E501EEF75F050A42435
:102B8D0000F9743235F0FA7BFF78247C007D007EED
:092B9D00007F501213FDC2192241
:102AB800900352E0C3941E502B122F20900352E033
:102AC80075F050A42400F582E5F03432AF82FE7B25
:102AD800007A0079249003D6E4F0A37450F0122908
:052AE800791219F02233
:062F4300122AB8C2192297
:05215D009003C8EDF045
:102162009003CAE004F09003CDEFF0A3EBF09003EC
:10217200C8E0FF9003CDE0FED39F4003022210751A
:10218200F050EEA42400F582E5F03432AF829003E1
:10219200CFF0A3EFF09003CEE075F050A42400F549
:1021A20082E5F03432AF829003D1F0A3EFF0E490F5
:1021B20003CBF0A3F09003D1E475F0011214F8AF51
:1021C200F0FE9003CFE0FCA3E0F5828C83E493FD64
:1021D2001225119003D0E004F070069003CFE004C2
:1021E200F09003CCE004F070069003CBE004F0C35F
:1021F2009003CCE094509003CBE0940040B71219C6
:0E220200F09003CDE004F0A3E004F0022170A0
:0122100022AB
:05175C009003C7EDF051
:101761009003CCEFF0A3EBF09003C7E0FF9003CC24
:10177100E0D39F40030218CDA3E075F050A42400EC
:10178100F582E5F03432AF829003C8F0A3EFF0E4C4
:101791009003CEF0A3F09003CEE0FEA3E0FFC3944C
:1017A10050EE940050389003C8E0FCA3E0F5828C21
:1017B10083E493FD74532FF582E43403F583EDF054
:1017C1009003C9E004F070069003C8E004F09003B0
:1017D100CFE004F070C09003CEE004F080B8900335
:1017E100CCE075F050A42400F582E5F03432AF82EC
:1017F1009003CAF0A3EFF09003CDE075F050A4245C
:1018010000F582E5F03432AF829003C8F0A3EFF027
:10181100E49003CEF0A3F09003C8E475F001121434
:10182100F8AFF0FE9003CAE0FCA3E0F5828C83E4FC
:1018310093FD1225119003CBE004F070069003CACA
:10184100E004F09003CFE004F070069003CEE004D2
:10185100F0C39003CFE094509003CEE0940040B7E2
:101861009003CCE075F050A42400F582E5F0343209
:10187100AF829003CAF0A3EFF0E49003CEF0A3F09F
:101881009003CEE0FCA3E0FDC39450EC9400502CF7
:101891009003CAE475F0011214F8AFF0FE74532DF1
:1018A100F582E43403F583E0FD1225119003CFE0C6
:1018B10004F070CC9003CEE004F080C41219F090D3
:0C18C10003CCE004F0A3E004F00217697F
:0118CD0022F8
:0B20A7009003C7EFF0A3EDF0A3EBF0F7
:1020B200A2AFE433A3F0C2AF122F2F9003C8E0FE09
:1020C2009003C7E0FDEDFF9003CFEEF0A3EFF0E445
:1020D2009003CBF09003C9E0FF9003CFE0FCA3E0B4
:1020E200FD7B017A0379539003D7E4F0A37450F097
:1020F200122BEE9003D0E02450F09003CFE0340096
:10210200F09003CBE075F050A42400F9743235F05E
:10211200FAA374FFF0A3EAF0A3E9F0122F209003D0
:10212200CCA3E0FAA3E0AE02FF7B017A03795390DD
:1021320003D6E4F0A37450F01229791219F0900337
:10214200CBE004F0E0C3941E408A9002A3E0FF12A9
:0A2152002EA99003CAE024FF92AF0B
:01215C002260
:0B235C009003C7EFF0A3EDF0A3EBF03F
:10236700A2AFE433A3F0C2AF122F2F9003C8E0FE51
:102377009003C7E0FDEDFF9003CCEEF0A3EFF0E490
:102387009003CBF09003CBE0FFC3941E504C75F045
:1023970050EFA42400F582E5F03432AF82FE9003BB
:1023A700CEF0FAA3EFF0FB9003C9E0FF9003CCE077
:1023B700FCA3E0FDA9037BFF9003D6E4F0A37450D0
:1023C700F0122D7F9003CDE02450F09003CCE03441
:1023D70000F09003CBE004F080AA9002A3E0FF1284
:0A23E7002EA99003CAE024FF92AF74
:0123F10022C9
:03000000020800F3
:03000300021A03DB
:03000B00021A06D0
:03001300021A09C5
:03001B00021A0CBA
:03002300021A0FAF
:03002B00021A12A4
:03003300021A1599
:03003B00021A188E
:03004300021A1B83
:03004B00021A1E78
:03005300021A216D
:03005B00021A2462
:03006300021A2757
:03006B00021A2A4C
:03007300021A2D41
:10080000E4F5D9E5EF7480F5FF7402F5EF787FE445
:10081000F6D8FD9000007F007E04E4F0A3DFFCDE4C
:07082000FA75817302086202
:100827000208A7E493A3F8E493A34003F68001F238
:1008370008DFF48029E493A3F85407240CC8C333D2
:10084700C4540F4420C8834004F456800146F6DFA1
:10085700E4800B0102040810204080902894E47E75
:10086700019360BCA3FF543F30E509541FFEE49396
:10087700A360010ECF54C025E060A840B8E493A35D
:10088700FAE493A3F8E493A3C8C582C8CAC583CA88
:10089700F0A3C8C582C8CAC583CADFE9DEE780BE40
:0128E10000F6
:10132D00E709F608DFFA8046E709F208DFFA803EA2
:10133D0088828C83E709F0A3DFFA8032E309F6088F
:10134D00DFFA8078E309F208DFFA807088828C83F7
:10135D00E309F0A3DFFA806489828A83E0A3F608AB
:10136D00DFFA805889828A83E0A3F208DFFA804C85
:10137D0080D280FA80C680D4806980F2803380105C
:10138D0080A680EA809A80A880DA80E280CA8033C5
:10139D0089828A83ECFAE493A3C8C582C8CCC5833D
:1013AD00CCF0A3C8C582C8CCC583CCDFE9DEE7800D
:1013BD000D89828A83E493A3F608DFF9ECFAA9F08C
:1013CD00EDFB2289828A83ECFAE0A3C8C582C8CCE2
:1013DD00C583CCF0A3C8C582C8CCC583CCDFEADEFB
:1013ED00E880DB89828A83E493A3F208DFF980CC5D
:1013FD0088F0EF60010E4E60C388F0ED2402B40456
:10140D000050B9F582EB2402B4040050AF232345FC
:06141D00822390137D7391
:10142300BB010689828A83E0225002E722BBFE02C7
:09143300E32289828A83E49322FA
:10143C00BB010CE58229F582E5833AF583E0225065
:10144C0006E92582F8E622BBFE06E92582F8E222AF
:0D145C00E58229F582E5833AF583E49322C9
:10146900BB010FF8E58229F582E5833AF583E02887
:10147900F0225009C58229F8E58226F622BBFE0929
:10148900C58229F8E22582F222F8EA2583F583E963
:0314990093282273
:10149C00BB010689828A83F0225002F722BBFE012F
:0214AC00F32229
:1014AE00F8BB010DE58229F582E5833AF583E8F074
:1014BE00225006E92582C8F622BBFE05E92582C820
:0214CE00F22208
:1014D000EF8DF0A4A8F0CF8CF0A428CE8DF0A42E30
:0214E000FE22EA
:1014E200C5F0F8A3E028F0C5F0F8E5821582700295
:0614F2001583E038F02232
:1014F800A3F8E0C5F025F0F0E582158270021583A7
:06150800E0C838F0E82203
:10150E00EB9FF5F0EA9E42F0E99D42F0E89C45F033
:01151E0022AA
:10151F00E8600FECC313FCED13FDEE13FEEF13FFAA
:03152F00D8F122CE
:0C153200ECF0A3EDF0A3EEF0A3EFF0222C
:10153E00A8828583F0D083D08212155512155512CC
:10154E001555121555E473E493A3C583C5F0C583F1
:10155E00C8C582C8F0A3C583C5F0C583C8C582C8F7
:01156E00225A
:10156F00D083D082F8E4937012740193700DA3A30B
:10157F0093F8740193F5828883E47374029368601F
:06158F00EFA3A3A380DF1F
:10159500EF4E6012EF60010EEDBB010B89828A836D
:1015A500F0A3DFFCDEFA2289F05007F709DFFCA97A
:0C15B500F022BBFEFCF309DFFCA9F022D1
:00000001FF
